:10000000E4C06FC2FDC0FCC0FBC0FAC0F9C0F8C0BC
:10001000F7C0F6C0F5C0F4C0F3C0F2C0F1C0F0C044
:10002000EFC0EEC0EDC0ECC0EBC0EAC0E9C0E8C074
:10003000E7C0E6C0040309041A03540069006C0019
:100040006C002000480061007200620061007500D1
:100050006D001A036900320063002D00740069000E
:100060006E0079002D00750073006200120110010E
:10007000FF000008030431C6050101020001090266
:1000800012000101008005090400000000000000CA
:100090000100FF8E6932632D74696E792D7573626C
:1000A000202D2028632920323030362062792054D8
:1000B000696C6C204861726261756D0A006E6F74C4
:1000C00020696E2061636B2073746174650A007728
:1000D00072697465206661696C65640A00646174A4
:1000E00061203D2025780A00657863656564732189
:1000F0000A007772697465202564206279746573DB
:100100002C202564206578700A006E6F7420696E5B
:100110002061636B2073746174650A0064617461AB
:10012000203D2025780A0065786365656473210A9F
:1001300000726561642025642062797465732C20E7
:100140002564206578700A00726571756573742086
:10015000666F722064656C617920256475730A008E
:100160005365747570202578202578202578202502
:10017000780A0049324320726561643A2061646400
:1001800072657373206572726F7220402025780A41
:100190000069326320257320617420307825303265
:1001A000782C206C656E203D2025640A004932437E
:1001B000206465766963652061742061646472659A
:1001C000737320307825780A000011241FBECFEF0A
:1001D000D4E0DEBFCDBF11E0A0E0B1E0E6E3F5E1A1
:1001E00002C005900D92AA31B107D9F711E0AAE13A
:1001F000B1E001C01D92A335B107E1F707D499C959
:10020000FFCEE9E6F0E0808183608083E89A08957C
:10021000FF920F931F93CF93DF9360913301662377
:1002200051F180913001CCE0D0E0C81BD109C95C0C
:10023000DE4F635080912F018D3279F080911A0149
:1002400087FD11C0CE0123D48F3F09F494C08823C9
:1002500009F48EC090E080E008C08AE58093010137
:10026000683009F4A7C090E880E090931A01809369
:100270000001109233018091010184FF26C080911A
:1002800000018F3F11F1182F8930A0F5811B809359
:10029000000180911A0180FD35C02BE4F22E8F5FA2
:1002A00080931A0187FD35C0112309F054C004E082
:1002B00084E291E0612F86D2183019F08FEF80939D
:1002C0000001F0922301009301019AE089B1847149
:1002D00059F49150D9F71092340110922E018FEFFA
:1002E00060E070E040E08DD2DF91CF911F910F91DF
:1002F000FF90089518E0811B8093000180911A01FE
:1003000080FFCBCF93ECF92E8F5F80931A0187FF8C
:10031000CBCFC0913101D091320186FD32C0112383
:1003200099F01150DE01E4E2F1E0412F50E01F5F4F
:100330009A012B5D3E4F8D918193E217F307D9F718
:100340004F5F5F4FC40FD51FD0933201C09331016F
:10035000012F0C5FADCF84E291E0612F4AD4182FBA
:10036000893008F4A4C08FEF809300010EE1A9CF7B
:1003700090E08FEF7ACF8EE18093010190E08FEFD4
:1003800074CF112309F311509E01A4E2B1E0612F53
:1003900070E01F5FAB014B5D5E4FF90184918D935F
:1003A0002F5F3F4FA417B507C1F76F5F7F4FC60F91
:1003B000D71FCACF8881807629F52CE231E01092D0
:1003C0002C018981882389F410922D013093320108
:1003D0002093310190E822E08F81882321F48E81DF
:1003E000821708F442CF822F40CF8530B9F0863093
:1003F000F1F0883031F18930A1F18A3059F190E87B
:1004000020E0EACFCE019DD4282F8F3F09F04DC0C8
:10041000888187FD09C08FEF90E027CF8A81809384
:10042000340190E820E0D8CF8E8190E01ECF8B8100
:10043000813031F18230D9F0833059F190EC20E0F5
:10044000CBCF86E391E0909332018093310190E825
:1004500021E0C2CF309332012093310190E821E0B6
:10046000BBCF8A818093360190E820E0B5CF8EE73C
:1004700090E0909332018093310190EC22E1ACCF77
:100480008CE690E0909332018093310190EC22E170
:10049000A3CF8A81882371F484E390E090933201A2
:1004A0008093310190EC24E097CF90E895CF082F0E
:1004B0000C5FFECE813061F0823009F0BFCF82E563
:1004C00090E0909332018093310190EC2AE184CF47
:1004D00088E390E0909332018093310190EC2AE11F
:1004E0007BCFCF93CFB7CF934C9BFECF4C9B09C014
:1004F0004C9B07C04C9B05C04C9B03C04C9B01C050
:100500009EC0DF93C0913001DD27C95CDE4F4C9B5C
:1005100002C0DF91EBCF2F930F931F9309B12FEF01
:1005200004FB20F94F933F9319B14FEF012704FBD0
:1005300021F93BE031C04E7F012F19B1216028C065
:10054000102F4D7F2260000009B129C04B7F24602D
:10055000012F000019B12BC019B1477F28602AC0B4
:100560004F7E09B120612CC04F7D19B120622FC090
:100570004F7B09B1206432C0422709B149934FEF44
:100580000000102714FB20F919B11471A9F1297F7B
:1005900091F2012704FB21F909B1237F89F231503F
:1005A000F0F1102714FB22F919B1277E79F2012707
:1005B00004FB23F92F7C81F209B1102714FB24F9E5
:1005C0002F7971F200C019B1012704FB25F92F73AF
:1005D00059F200C009B1102714FB26F9223040F26D
:1005E00000C019B1012704FB27F9243028F64F7702
:1005F000206819B10000F9CF3B503195333011E03C
:100600001CBBB8F0C31BD0400881033C41F10B3444
:1006100031F11981412F1F7720912E01121731F4EA
:10062000093691F10D3279F0013E69F022272093CD
:1006300035013F914F911F910F912F91DF91CF91F4
:10064000CFBFCF911895009335013F914F911F91E6
:100650000F912F91DF91CCB3C0FD46CFF0CF009129
:100660003501002331F310913301112349F5343062
:100670004AF13093330100932F01109130013BE098
:10068000311B309330011EC0009133010130C4F49E
:100690000AE53091010134FD17C000930101C3E266
:1006A000D1E016C0052710E00BB91FC0052722C0F6
:1006B000052727C005272CC0052710E00BB933C03C
:1006C0004AE503C042ED01C0432FC4E1D0E032E06F
:1006D0001AB114615C9A0BB11AB95F9354E120E826
:1006E00020FF05270BB9279517951C3FD8F620FF4B
:1006F000052727950BB917951C3FC0F620FF052746
:10070000279517950BB91C3F98F620FF05272795CD
:1007100017951C3F0BB970F600C0499120FF0527C3
:100720000BB9279517951C3F38F620FF052727950D
:100730000BB917951C3F38F520FF0527279517950E
:100740000BB91C3F10F520FF0527279517951C3F77
:100750000BB9E8F4242F3A9519F60B7E5F910BB98B
:1007600000C010913401C651D04011F010932E01F9
:1007700011E01CBB00611AB11B7E402F4B7E0BB9F0
:100780001AB94BB956CF0527D3CF0527D8CF0527A0
:10079000DDCFA82FB92F8FEF9FEF41E050EA6150D6
:1007A00070F02D9138E0722F7827969587952695D1
:1007B00070FF02C0842795273A95A9F7F0CF80955E
:1007C00090950895E6DF8D939D930895282F982F97
:1007D00092959F709A3008F0995D8091C00085FFD6
:1007E000FCCF905D9093C600922F9F709A3008F0D6
:1007F000995D8091C00085FFFCCF905D9093C6000D
:100800000895FF920F931F93CF93DF93062FF72E38
:10081000142FDCDF8091C00085FFFCCF8AE380933A
:10082000C6001123B9F01150802F9F2DEC0180E2FA
:10083000F82ECE01810F911D8C018091C00085FFA3
:10084000FCCFF092C6008881C1DFC017D10711F03C
:100850002196F3CF8091C00085FFFCCF8DE080937F
:10086000C6008091C00085FFFCCF8AE08093C6005F
:10087000DF91CF911F910F91FF9008951F93182F33
:100880008A3051F08091C00085FFFCCF1093C600E4
:1008900080E090E01F9108958DE0F0DFF3CF882392
:1008A00019F43C9A449808953C98449A0895E0912C
:1008B0001801F09119013197F1F7882359F03D980B
:1008C000459A359BFECF80911601909117010197B3
:1008D000F1F708953D9A4598F6CF81E0E8DF80E092
:1008E000E6DF089580E0DBDF80E0E1DF089580E06F
:1008F000D6DF81E0DCDF81E0D2DF08950F931F9324
:10090000CF93DF93082F10E0C7E0D0E008C081E06C
:10091000C6DFE3DF21978FEFCF3FD80789F0C8010B
:100920000C2E02C0959587950A94E2F780FDEFCFD3
:1009300080E0B5DFD2DF21978FEFCF3FD80779F77F
:1009400081E0ADDF81E0B3DF16B180E0B0DF12956A
:100950001F701095812F8170DF91CF911F910F91A2
:100960000895FF920F931F93F82E81E098DF80E0A7
:100970009EDF17E000E081E09ADF000F349901600C
:1009800080E095DF1150B8F7FF2051F480E087DF59
:10099000A4DF81E084DF802F1F910F91FF900895E5
:1009A00081E07DDF9ADF81E07ADF802F1F910F9158
:1009B000FF9008950F931F93CF93DF93C0E0D0E093
:1009C0000DEA11E005C093DF2196CF37D105C9F0BC
:1009D00089DF9E01220F822F91DF8823A1F300D0AF
:1009E00000D0EDB7FEB712830183D483C383D9D27D
:1009F0000F900F900F900F907ADF2196CF37D1058F
:100A000039F7DF91CF911F910F9108952EE088E182
:100A100090E00FB6F894A895809360000FBE2093E5
:100A200060008091C10088608093C10082E090E006
:100A30009093C5008093C40088E091E090935001AA
:100A400080934F0100D084E990E0EDB7FEB7928328
:100A50008183A7D23C98449A3D98459A10922101EF
:100A6000109220010F900F90A5DF8BB18B7E8BB978
:100A70008AB184618AB980E49CE90197F1F78AB16F
:100A80008B7E8AB9BEDB7894A895C2DBFDCFDF925E
:100A9000EF92FF920F931F93CF93DF93D82E092FDE
:100AA000162F00D000D000D0EDB7FEB7319682EF00
:100AB00090E0ADB7BEB712969C938E931197628368
:100AC000138280912001909121019583848369D2C2
:100AD000EDB7FEB736960FB6F894FEBF0FBEEDBF6A
:100AE00080911B01813009F054C0212F30E08091AA
:100AF0002001909121018217930708F464C011230B
:100B000009F475C08D2D902F9C01E90100E08DED59
:100B1000E82E80E0F82E809120019091210101972C
:100B2000909321018093200100D000D0EDB7FEB753
:100B30003196ADB7BEB71296FC92EE9211978881AE
:100B4000828313822ED20F900F900F900F90899175
:100B5000D5DE882309F401E0FE01ED19E117D8F292
:100B60008091220181FF06C0809120019091210196
:100B7000892BD9F10023F1F000D08FEC90E0ADB7D4
:100B8000BEB712969C938E9311970BD20F900F9035
:100B900011C000D08DEB90E0EDB7FEB7928381835A
:100BA00000D20F900F908D2D902F60E070E0412FBC
:100BB00050E0F0D1812FDF91CF911F910F91FF90E5
:100BC000EF90DF90089500D088EE90E0ADB7BEB70B
:100BD00012969C938E931197E4D1109120010F905F
:100BE0000F90112309F08ECF02C081DEC3CF00E049
:100BF000B7CFEF92FF920F931F93CF93DF93082FFE
:100C0000F92E162F00D000D000D0EDB7FEB73196E8
:100C100081E391E0ADB7BEB712969C938E93119786
:100C200062831382809120019091210195838483B6
:100C3000B8D1EDB7FEB736960FB6F894FEBF0FBE2B
:100C4000EDBF80911B01813009F04CC0212F30E0B5
:100C500080912001909121018217930708F45DC0D3
:100C6000112371F1802F9F2D9C01E9019CE1E92E58
:100C700091E0F92E809120019091210101979093AC
:100C800021018093200120E0892B09F421E0822FAB
:100C900068DE899300D000D0EDB7FEB73196ADB7CE
:100CA000BEB71296FC92EE9211978283138279D18D
:100CB000FE01E01B0F900F900F900F90E117D0F204
:100CC0008091220181FF06C0809120019091210135
:100CD000892BA9F1812FDF91CF911F910F91FF9067
:100CE000EF90089500D08AE091E0ADB7BEB71296BC
:100CF0009C938E93119755D10F900F90802F9F2D1D
:100D000060E070E0412F50E045D1812FDF91CF911D
:100D10001F910F91FF90EF90089500D087E291E02E
:100D2000ADB7BEB712969C938E9311973AD110919E
:100D300020010F900F90112309F094CFC1CFD7DD80
:100D4000C9CF0F931F93CF93DF93EC010CE111E018
:100D500010933201009331012DB73EB72A50304035
:100D60000FB6F8943EBF0FBE2DBFEDB7FEB731965C
:100D700080E691E0ADB7BEB712969C938E93119723
:100D80008881828313828981848315828A81868304
:100D900017828B818087118604D1EDB7FEB73A9612
:100DA0000FB6F894FEBF0FBEEDBF8981823009F403
:100DB00079C0833008F44FC0833009F4A3C0883071
:100DC00008F05EC08A8180FDB1C022E031E0EDB75D
:100DD000FEB738970FB6F894FEBF0FBEEDBF319641
:100DE00081E991E0ADB7BEB712969C938E931197AF
:100DF000338322838C819D81958384838E819F811F
:100E000097838683CED01C81110F8A81EDB7FEB700
:100E100038960FB6F894FEBF0FBEEDBF80FD11608F
:100E2000898180FF86C05EDD812F68DD882309F41B
:100E300089C081E080931B012E813F813093210185
:100E40002093200189818093220181FF17C0232BE9
:100E500091F08FEF16C08823C9F0813089F4C80162
:100E600060E970E044E050E08CD084E0DF91CF9105
:100E70001F910F9108953BDD2E813F81232B49F770
:100E800080E0DF91CF911F910F9108958A81809327
:100E90001C018B8180931D0182E0DF91CF911F9116
:100EA0000F9108952A813B813093170120931601F9
:100EB0002115310589F581E090E090931701809329
:100EC000160121E030E081E090E0909319018093D9
:100ED000180100D000D088E491E0ADB7BEB71296FB
:100EE0009C938E93119714963C932E93139759D0FD
:100EF00080E00F900F900F900F90DF91CF911F9196
:100F00000F91089580911B0180931C0181E0DF9176
:100F1000CF911F910F910895C90196958795909350
:100F2000190180931801892BA1F6CDCF25E031E07E
:100F30004ECF81E0B4DC81E0BADC80E0B0DC80E060
:100F4000B6DC72CF00D000D0EDB7FEB7319683E7A4
:100F500091E0ADB7BEB712969C938E931197128312
:100F600013821FD082E080931B0110922101109206
:100F700020010F900F900F900F90B9DC2E813F81D0
:100F80007DCFFB01DC0102C005900D924150504025
:100F9000D8F70895DC0101C06D9341505040E0F74F
:100FA0000895A0E0B0E0E6EDF7E09CC2FE013596C2
:100FB00061917191A0914F01B091500113968C9164
:100FC0001397886013968C9380914F0190915001F4
:100FD000AF010AD0E0914F01F09150012381277FAA
:100FE00023832096E2E09AC2ABE0B0E0E9EFF7E0BD
:100FF00069C23C012B015A01FC01178216828381D0
:1010000081FD03C06FEF7FEFB9C19AE0892E1E0109
:101010000894211C311CF3012381F20123FD8591E9
:1010200023FF81912F01882309F4A5C1853239F46A
:1010300023FD859123FF81912F01853221F490E0DA
:10104000B301B6D1E8CF982FFF24EE249924FFE115
:10105000FF15D0F09B3269F09C3228F4903259F0A1
:10106000933291F40EC09D3249F0903369F441E01F
:1010700024C052E0F52A84E0F82A28C098E0F92A32
:1010800025C0E0E1FE2A22C0F7FC29C0892F805349
:101090008A3070F4F6FE05C0989C902C1124980EAE
:1010A00015C0E89CE02C1124E80EF0E2FF2A0EC0E7
:1010B0009E3229F4F6FC5FC140E4F42A07C09C3656
:1010C00019F450E8F52A02C0983649F4F20123FDDC
:1010D000959123FF91912F01992309F0B8CF892F82
:1010E0008554833018F08052833038F444E050E067
:1010F000A40EB51E5FE359830FC0933631F09337CA
:1011000079F0933509F052C01FC0F50180818983C1
:1011100042E050E0A40EB51E610101E010E011C0F4
:10112000F501C080D180F6FC03C06FEF7FEF02C0F5
:10113000692D70E042E050E0A40EB51EC6012DD12D
:101140008C015FE7F52213C0F501C080D180F6FC69
:1011500003C06FEF7FEF02C0692D70E042E050E006
:10116000A40EB51EC6010ED18C0150E8F52AF3FE7F
:1011700006C018C080E290E0B3011AD1EA948E2D27
:1011800090E008171907B0F30DC0F601F7FC859140
:10119000F7FE81916F0190E0B3010AD1E110EA946A
:1011A000015010400115110581F7E2C0943611F08D
:1011B000993661F5F7FE08C0F50120813181428141
:1011C000538184E090E00AC0F501808191819C0107
:1011D000442737FD4095542F82E090E0A80EB91EB9
:1011E0009FE6F92257FF09C050954095309521950B
:1011F0003F4F4F4F5F4FE0E8FE2ACA01B901A101FE
:101200002AE030E001D1D82ED2183FC0953729F41A
:101210001F2D1F7E2AE030E01DC01F2D197F9F3635
:1012200061F0903720F4983509F0A5C00FC09037D1
:1012300039F0983709F09FC004C028E030E00AC0B8
:10124000106114FD146020E130E004C014FD16604C
:1012500020E132E017FF08C0F501608171818281D1
:10126000938144E050E008C0F50180819181BC0188
:1012700080E090E042E050E0A40EB51EA101C4D091
:10128000D82ED2188FE7F82EF122F6FE0BC05EEFB3
:10129000F522D91438F4F4FE07C0F2FC05C08FEE35
:1012A000F82202C01D2D01C0192DF4FE0DC0FE0153
:1012B000ED0DF11D8081803319F499EEF92208C0FB
:1012C0001F5FF2FE05C003C08F2D867809F01F5FF7
:1012D0000F2DF3FC13C0F0FE0EC01E1510F09D2C58
:1012E0000AC09D2C9E0C911A1E2D05C080E290E034
:1012F000B3015ED01F5F1E15C8F304C01E1510F4A5
:10130000E11A01C0EE2404FF0EC080E390E0B301B7
:101310004FD002FF1BC001FD03C088E790E00EC064
:1013200088E590E00BC0802F867881F001FF02C035
:101330008BE201C080E2F7FC8DE290E0B30138D08F
:1013400005C080E390E0B30133D09A94D914C8F378
:10135000DA94F101ED0DF11D808190E0B30128D008
:10136000DD20B1F705C080E290E0B30121D0EA941E
:10137000EE20C9F750CEF30166817781CB012B9621
:10138000E2E1BCC0FC010590615070400110D8F74B
:10139000809590958E0F9F1F0895FC0161507040BD
:1013A00001900110D8F7809590958E0F9F1F08959A
:1013B0000F931F93CF93DF938C01EB018B8181FF00
:1013C0001BC082FF0DC02E813F818C819D8128171B
:1013D000390764F4E881F9810193F983E88306C051
:1013E000E885F985802F0995892B31F48E819F81BD
:1013F00001969F838E8302C00FEF1FEFC801DF911C
:10140000CF911F910F910895FA01AA27283051F129
:10141000203181F1E8946F936E7F6E5F7F4F8F4F25
:101420009F4FAF4FB1E03ED0B4E03CD0670F781F84
:10143000891F9A1FA11D680F791F8A1F911DA11D69
:101440006A0F711D811D911DA11D20D009F46894A2
:101450003F912AE0269F11243019305D3193DEF64A
:10146000CF010895462F4770405D4193B3E00FD000
:10147000C9F7F6CF462F4F70405D4A3318F0495DEB
:1014800031FD4052419302D0A9F7EACFB4E0A695CE
:101490009795879577956795BA95C9F700976105F0
:1014A000710508959B01AC010A2E06945795479546
:1014B00037952795BA95C9F7620F731F841F951F3B
:1014C000A01D08952F923F924F925F926F927F924C
:1014D0008F929F92AF92BF92CF92DF92EF92FF9244
:1014E0000F931F93CF93DF93CDB7DEB7CA1BDB0BF0
:1014F0000FB6F894DEBF0FBECDBF09942A88398895
:1015000048885F846E847D848C849B84AA84B9849B
:10151000C884DF80EE80FD800C811B81AA81B981A7
:10152000CE0FD11D0FB6F894DEBF0FBECDBFED01BB
:061530000895F894FFCFBE
:10153600FF5A77720072640000000002000000008B
:0A1546003E04000000000A0005004A
:00000001FF
